:020000040000FA
:0600000000308A007228A6
:08000800F000030E8301F1007A
:100010000A08F2008A0183130408F30083168C1A7D
:1000200013288312582883128C1E5828861387148D
:10003000071476158E018F010C1083160C14831291
:100040001A08F70098185428181D2D281812181689
:100050007614F501F401F8010E28761C0E28F40838
:10006000031D3B28F508031D3B28F61026087706DC
:100070000319F6145028F61C0E287808103A0319B4
:10008000502825087502F90024087402031CF9039E
:10009000F91B50282E307807840077088000F80A72
:1000A000F40A0319F50A0E281812181607120E285A
:1000B00083160C185D288312692883120C1C69288A
:1000C0000C1083160C1083128617871007107611F8
:1000D0000E287308840072088A00710E8300F00EE7
:1000E000700E090085018601870183161030850096
:1000F0000F308600CC30870007309F008312051137
:1001000085108516851505140510051486178710AA
:10011000071007168716061686160617A1012E3039
:1001200084008001840AA10A2108103A031D912845
:10013000F601F501F401F801A201071D22140613CE
:10014000000006090F39A9000617000086120000FA
:1001500006090F39AA0086160000061200000609DB
:100160000F39AB0006161821AD080319C5282D0854
:10017000013C031CC0282C08F13C031CC228CA28DF
:100180000130AD00F130AC00CA28AC08031DCA280C
:100190000130AC002C08A4002D08A5000030A600FA
:1001A000831604309900181518128C16831218172C
:1001B000181698179001901610148B010B178B17B7
:1001C000A0012E30840003100530A100A00DA10B6A
:1001D000E6280330A100A00D051103180515000045
:1001E000851400008510A10BEB28A00D0008A300CA
:1001F0002218A30903100830A100A30D051103184C
:1002000005150000851400008510A10BFD28A30D25
:10021000A0190E29851200008516112985110000EC
:100220008515A00A840A2008103A031DE328E02857
:10023000AD012908AC0024212A08AC0724212B0891
:10024000AC070318AD0A08002C08A7002D08A80069
:100250000310AC0DAD0D0310AC0DAD0D2708AC07B0
:10026000031C3329AD0A2808AD070310AC0DAD0DF2
:02027000080084
:02400E00723FFF
:00000001FF
